:100000000C9462000C948A000C948A000C948A0070
:100010000C948A000C948A000C948A000C948A0038
:100020000C948A000C948A000C948A000C948A0028
:100030000C948A000C948A000C948A000C948A0018
:100040000C9497010C948A000C940D030C948A0074
:100050000C948A000C948A000C948A000C948A00F8
:100060000C948A000C948A000000000024002700F1
:100070002A0000000000250028002B0000000000DE
:1000800023002600290004040404040404040202DA
:100090000202020203030303030301020408102007
:1000A0004080010204081020010204081020000012
:1000B0000007000201000003040600000000000029
:1000C0000000920411241FBECFEFD8E0DEBFCDBFE9
:1000D00011E0A0E0B1E0E4ECFCE002C005900D927C
:1000E000AA31B107D9F711E0AAE1B1E001C01D9230
:1000F000AF3BB107E1F710E0C4ECD0E004C02297B9
:10010000FE010E945C06C23CD107C9F70E94900123
:100110000C9460060C940000809106010E94BE02BF
:10012000892B39F48CEA91E040E050E060E070E027
:100130000CC0809106010E94BE02892B51F08CEA0E
:1001400091E041E050E060E070E020E030E00E94AB
:10015000C20580910A010E94BE02892B09F043C0AA
:100160008CEA91E042E050E060E070E020E030E0B6
:100170000E94C2050E94DF0120911C0130911D01E7
:10018000442737FD4095542F621B730B840B950B4E
:100190002091000130910101442737FD4095542FF3
:1001A000261737074807590770F50E94DF0170933B
:1001B0001D0160931C0180911A0190911B01892BF4
:1001C00039F481E090E090931B0180931A0104C000
:1001D00010921B0110921A018091040160911A0182
:1001E0000E94710210C080910A010E94BE02892BF8
:1001F00051F08CEA91E043E050E060E070E020E0F4
:1002000030E00E94C20564E670E080E090E00E9469
:10021000ED018CEA91E00E944304882331F18CEADD
:1002200091E00E94570480931E01803121F4809157
:10023000020161E005C0803231F48091020160E08A
:100240000E9471020895803381F480910C0161E075
:100250000E94710264E670E080E090E00E94ED018F
:1002600080910C0160E00E94710208958CEA91E097
:1002700040E05BE460E070E00E944A03809102018C
:1002800061E00E9451028091060160E00E945102EB
:100290008091040161E00E94510280910A0160E0B6
:1002A0000E9451028091080161E00E9451028091F8
:1002B0000C0161E00E94510280910E0161E00E94F8
:1002C00051028091020160E00E947102809106015A
:1002D00061E00E9471028091040161E00E9471025C
:1002E00080910A0161E00E9471028091080160E042
:1002F0000E94710280910E0160E00E947102809163
:100300000C0161E00E94710264E670E080E090E020
:100310000E94ED0180910C0160E00E94710208953D
:100320000E9417020E9436010E948C00FDCF1F928E
:100330000F920FB60F9211242F933F938F939F9399
:10034000AF93BF938091230190912401A091250147
:10035000B0912601309127010196A11DB11D232FD7
:100360002D5F2D3720F02D570196A11DB11D209333
:1003700027018093230190932401A0932501B0933A
:10038000260180911F0190912001A0912101B0913F
:1003900022010196A11DB11D80931F0190932001A0
:1003A000A0932101B0932201BF91AF919F918F91B2
:1003B0003F912F910F900FBE0F901F9018958FB700
:1003C000F89420912301309124014091250150910E
:1003D00026018FBFB901CA010895EF92FF920F93D2
:1003E0001F937B018C018FB7F894409123015091AA
:1003F000240160912501709126018FBF2FB7F894D9
:100400008091230190912401A0912501B0912601B2
:100410002FBF841B950BA60BB70BE816F9060A072E
:100420001B0760F71F910F91FF90EF90089578944C
:1004300084B5826084BD84B5816084BD85B58260E9
:1004400085BD85B5816085BDEEE6F0E08081816087
:100450008083E1E8F0E08081826080838081816038
:100460008083E0E8F0E0808181608083E1EBF0E070
:10047000808184608083E0EBF0E080818160808314
:10048000EAE7F0E0808184608083808182608083FD
:100490008081816080838081806880831092C10028
:1004A0000895282F30E0C90186569F4FFC01949192
:1004B0002A573F4FF9018491882391F0E82FF0E00B
:1004C000EE0FFF1FE859FF4FA591B491662329F461
:1004D0008C91909589238C9308958C91892B8C9382
:1004E0000895482F50E0CA0182559F4FFC01249186
:1004F000CA0186569F4FFC0194914A575F4FFA01FB
:1005000034913323D1F1222331F1233021F480912E
:1005100080008F7705C0243031F4809180008F7D7A
:100520008093800018C0213019F484B58F7704C0FF
:10053000223021F484B58F7D84BD0DC0263021F496
:100540008091B0008F7705C0273029F48091B000EA
:100550008F7D8093B000E32FF0E0EE0FFF1FEE5889
:10056000FF4FA591B491662329F48C91909589232E
:100570008C9308958C91892B8C930895682F70E04B
:10058000CB0182559F4FFC012491CB0186569F4F92
:10059000FC0144916A577F4FFB019491992319F410
:1005A00020E030E038C0222331F1233021F4809163
:1005B00080008F7705C0243031F4809180008F7DDA
:1005C0008093800018C0213019F484B58F7704C05F
:1005D000223021F484B58F7D84BD0DC0263021F4F6
:1005E0008091B0008F7705C0273029F48091B0004A
:1005F0008F7D8093B000892F90E0880F991F8458D9
:100600009F4FFC01A591B4918C9120E030E08423B0
:1006100011F021E030E0C90108951F920F920FB64A
:100620000F9211242F933F934F935F936F937F9378
:100630008F939F93AF93BF93EF93FF934091C60027
:10064000E091A801F091A901CF01019660E870E066
:100650000E94F6059C018091AA019091AB01281798
:10066000390739F0E85DFE4F40833093A9012093AC
:10067000A801FF91EF91BF91AF919F918F917F91D1
:100680006F915F914F913F912F910F900FBE0F90FF
:100690001F9018955F926F927F928F929F92AF9268
:1006A000BF92CF92DF92EF92FF920F931F93CF935F
:1006B000DF93EC013A014B01413482E458078FE0AB
:1006C000680780E078070CF07FC060E874E88EE18E
:1006D00090E0A40193010E942B062150304040403D
:1006E0005040CA01B90122E030E040E050E00E94F1
:1006F0002B0659016A01A601950120953095409578
:10070000509594E0220F331F441F551F9A95D1F73F
:1007100060E074E284EF90E00E942B06CA01B90108
:100720002FEF30E040E050E00E94D705A401930194
:100730000E942B06C90181509F4F181619061CF400
:10074000522E5A9403C055245394521A60E079E013
:100750008DE390E0A40193010E942B0621503040CC
:1007600040405040CA01B90122E030E040E050E092
:100770000E942B06209530954095509583E0220FDE
:10078000331F441F551F8A95D1F760E074E284EF50
:1007900090E00E942B06CA01B9012FEF30E040E043
:1007A00050E00E94D705A40193010E942B06C901C5
:1007B00081509F4F181619061CF4822F815002C0D9
:1007C00081E0821B851500F5E885F98581E090E0E0
:1007D0000A8802C0880F991F0A94E2F7808360E0BC
:1007E00079E08DE390E0A40193010E942B06215053
:1007F000304040405040CA01B90122E030E040E0C2
:1008000050E00E942B0604C0E885F985108295010E
:10081000EC81FD813083EE81FF812083EA85FB85B9
:10082000208141E050E0CA010E8402C0880F991F68
:100830000A94E2F7282B2083EA85FB852081CA01F0
:100840000F8402C0880F991F0A94E2F7282B208397
:10085000EA85FB858081088802C0440F551F0A94F1
:10086000E2F7842B8083DF91CF911F910F91FF904E
:10087000EF90DF90CF90BF90AF909F908F907F9040
:100880006F905F900895DC011296ED91FC911397A3
:10089000E058FF4F8191919180589F4F2081318185
:1008A000821B930B60E870E00E94F6050895CF93D9
:1008B000DF93DC011296ED91FC911397EF01CE5777
:1008C000DF4F48815981E058FF4F80819181E05886
:1008D000F0408417950719F42FEF3FEF0CC0E40F99
:1008E000F51F2081CA01019660E870E00E94F605BC
:1008F0009983888330E0C901DF91CF910895FC018D
:10090000A085B18521898C9190E0022E02C0959539
:1009100087950A94E2F780FFF6CF0484F585E02DF1
:100920006083089584E191E09093AD018093AC01E0
:1009300088E291E09093AF018093AE0185EC90E066
:100940009093B1018093B00184EC90E09093B30157
:100950008093B20180EC90E09093B5018093B40154
:1009600081EC90E09093B7018093B60186EC90E023
:100970009093B9018093B80184E08093BA0183E039
:100980008093BB0187E08093BC0185E08093BD012B
:1009900081E08093BE0108950F931F93CF93DF935F
:1009A0008C01EB0109C02196D801ED91FC910190D9
:1009B000F081E02DC801099568816623A1F7DF91D8
:1009C000CF911F910F910895EF92FF920F931F9374
:1009D000CF93DF938C017B01EA010CC0D7016D91AD
:1009E0007D01D801ED91FC910190F081E02DC801CD
:1009F00009952197209791F7DF91CF911F910F9142
:100A0000FF90EF9008952F923F924F925F926F92D6
:100A10007F928F929F92AF92BF92CF92DF92EF928E
:100A2000FF920F931F93DF93CF93CDB7DEB7A097BD
:100A30000FB6F894DEBF0FBECDBF1C016A017B016B
:100A4000411551056105710549F4DC01ED91FC91F9
:100A50000190F081E02D60E3099554C08824992429
:100A60005401422E55246624772401E010E00C0F37
:100A70001D1F080D191DC701B601A30192010E9497
:100A80000906F80160830894811C911CA11CB11C0B
:100A9000C701B601A30192010E940906C901DA014A
:100AA0006C017D01C114D104E104F104F1F681E08F
:100AB000E82EF12CEC0EFD1EE80CF91C3E0108940A
:100AC000611C711CD501C4010197A109B1096C0118
:100AD000C818D90814C0F601EE0DFF1D60816A30F8
:100AE00010F4605D01C0695CD101ED91FC91019051
:100AF000F081E02DC10109950894E108F1086E1418
:100B00007F0449F7A0960FB6F894DEBF0FBECDBFA5
:100B1000CF91DF911F910F91FF90EF90DF90CF90D9
:100B2000BF90AF909F908F907F906F905F904F900D
:100B30003F902F900895EF92FF920F931F93CF93C2
:100B4000DF93EC017A018B0177FF0FC0E881F98117
:100B50000190F081E02D6DE2099510950095F094DB
:100B6000E094E11CF11C011D111DCE01B801A7018B
:100B70002AE00E940305DF91CF911F910F91FF9012
:100B8000EF900895DC012115310541F4ED91FC91C0
:100B90000190F081E02D642F099508952A303105E8
:100BA00019F40E949B0508950E9403050895629F11
:100BB000D001739FF001829FE00DF11D649FE00D55
:100BC000F11D929FF00D839FF00D749FF00D659FB6
:100BD000F00D9927729FB00DE11DF91F639FB00DB5
:100BE000E11DF91FBD01CF011124089597FB092EC6
:100BF00007260AD077FD04D049D006D000201AF489
:100C0000709561957F4F0895F6F7909581959F4F68
:100C10000895A1E21A2EAA1BBB1BFD010DC0AA1F3D
:100C2000BB1FEE1FFF1FA217B307E407F50720F055
:100C3000A21BB30BE40BF50B661F771F881F991FD0
:100C40001A9469F760957095809590959B01AC0119
:100C5000BD01CF01089597FB092E05260ED057FD43
:100C600004D0D7DF0AD0001C38F450954095309559
:100C700021953F4F4F4F5F4F0895F6F79095809520
:100C8000709561957F4F8F4F9F4F0895AA1BBB1B97
:100C900051E107C0AA1FBB1FA617B70710F0A61B7C
:100CA000B70B881F991F5A95A9F780959095BC019D
:100CB000CD010895EE0FFF1F0590F491E02D0994EA
:040CC000F894FFCFD6
:100CC400E8030A000E000F001000110008000900DC
:0A0CD400000000007F04CC04E404DB
:00000001FF
